S02B0000433A2F576F726B2F736F6674776172652F4F70656E424C542F5461726765742F44656D6F2F41524DEF
S31508006000F0010020FB610008B1650008B1650008D1
S31508006010B1650008B1650008B1650008B1650008FA
S31508006020B1650008B1650008B1650008B1650008EA
S31508006030B1650008B1650008B165000895650008F6
S31508006040B1650008B1650008B1650008B1650008CA
S31508006050B1650008B1650008B1650008B1650008BA
S31508006060B1650008B1650008B1650008B1650008AA
S31508006070B1650008B1650008B1650008B16500089A
S31508006080B1650008B1650008B1650008B16500088A
S31508006090B1650008B1650008B1650008B16500087A
S315080060A0B1650008B1650008B1650008B16500086A
S315080060B0B1650008B1650008B1650008B16500085A
S315080060C0B1650008B1650008B1650008B16500084A
S315080060D0B1650008B1650008B1650008B16500083A
S315080060E0B1650008B1650008B1650008B16500082A
S315080060F0B1650008B1650008B1650008B16500081A
S31508006100B1650008B1650008B1650008B165000809
S31508006110B1650008B1650008B1650008B1650008F9
S31508006120B1650008B1650008B1650008B1650008E9
S31508006130B1650008B1650008B1650008B1650008D9
S31508006140B1650008B1650008B1650008B1650008C9
S30908006150EE11AA553F
S315080061542B49072291438D462A482B492B4A00F09E
S3150800616439F82B482B492C4A00F034F82B482C498B
S315080061742C4A00F02FF82C482C492D4A00F02AF80E
S315080061842C482D492D4A00F025F82D482D492E4A2C
S3150800619400F020F82D482E49002200F026F82D4854
S315080061A42D49091A082903DB00220260043001601C
S315080061B41E481F49884205D00268043003B4904734
S315080061C403BCF7E700208646EC4600200021234A54
S315080061D49047FEE7884207D0521A05D00378013063
S315080061E40B700131013AF9D17047884202D0027026
S315080061F40130FAE770471A481A490160A8E700000F
S31508006204F001002044760008000000201400002055
S315080062146C6200086C620008207600084476000860
S3150800622400000020000000202076000820760008E0
S3150800623420760008207600082076000820760008D4
S31508006244207600082076000844760008140000200A
S315080062546D00002070000020F00000202163000873
S30D0800626408ED00E000600008E7
S3150800626C80B582B000AF012110200B4B98474FF434
S3150800627C8053BB800323BB711023FB713B1D19464E
S3150800628C0648074B98474FF480510448054B9847E6
S3150800629C00BF0837BD4680BD5D730008001001407D
S315080062AC6D6F0008E570000880B582B000AF134B1F
S315080062BC98477860124B1B687A68D31AB3F5FA7F3D
S315080062CC18D3104B1B78002B08D10E4B01221A70D1
S315080062DC4FF480510C480D4B984707E0094B0022A8
S315080062EC1A704FF480510848094B9847044A7B6842
S315080062FC136000E000BF0837BD4680BD8165000805
S3150800630C140000201800002000100140017100083C
S3150800631CE570000880B500AF044B9847044B9847C6
S3150800632C044B9847044B9847FAE700BF49630008A3
S3150800633CE1650008B5620008F965000880B584B007
S3150800634C00AF0023BB6000237B604F4A4E4B1B6893
S3150800635C43F0010313604C494B4B5A684B4B1340A3
S3150800636C4B60494A484B1B6823F0847323F48033EB
S3150800637C1360454A444B1B6823F480231360424A36
S3150800638C414B5B6823F4FE0353603F4B4FF41F02EB
S3150800639C9A603D4A3C4B1B6843F4803313603A4B76
S315080063AC1B6803F400337B60BB680133BB607B68F6
S315080063BC002B04D1BB6840F2DC529342EFD1324B2E
S315080063CC1B6803F40033002B00D1FEE7304A304B30
S315080063DC1B6843F0100313602D4A2D4B1B6823F0E2
S315080063EC030313602A4A2A4B1B6843F00203136003
S315080063FC254A254B5B685360234A234B5B6843F459
S3150800640C00535360204A204B5B6843F48063536007
S3150800641C1D4A1D4B5B6823F47C1353600923FB60F0
S3150800642CFB68023B9B04FB601749174B5A68FB68D1
S3150800643C134343F480334B60134A134B1B6843F0E6
S3150800644C8073136000BF104B1B6803F00073002B9E
S3150800645CF9D00D4A0C4B5B6823F0030353600A4AC8
S3150800646C094B5B6843F00203536000BF064B5B683D
S3150800647C03F00C03082BF9D1064B9847064B9847A3
S3150800648C00BF1037BD4680BD001002400000FFF863
S3150800649C002002406D6200084565000880B483B090
S315080064AC00AF03463960FB7197F90730002B0BDAFE
S315080064BC0D49FB7903F00F03043B3A68D2B212017B
S315080064CCD2B20B441A7609E0084997F907303A68AC
S315080064DCD2B21201D2B20B4483F8002300BF0C3798
S315080064ECBD4680BC704700BF00ED00E000E100E04F
S315080064FC80B582B000AF78607B68B3F1807F01D33A
S3150800650C012311E00A4A7B6823F07F43013B536061
S3150800651C0F214FF0FF30074B9847054B00229A6026
S3150800652C034B07221A60002318460837BD4680BD60
S3150800653C10E000E0A964000880B500AF0348044BDE
S3150800654C98470020034B984700BF80BD40190100AF
S3150800655CFD6400086565000880B483B000AF7860F8
S3150800656C034A7B68136000BF0C37BD4680BC704776
S3150800657C1C00002080B400AF024B1B681846BD46B1
S3150800658C80BC70471C00002080B400AF044B1B680D
S3150800659C0133034A136000BFBD4680BC704700BF79
S315080065AC1C00002080B400AFFEE700BF80B400AF2B
S315080065BCBFF34F8F0549054BDB6803F4E062044BC8
S315080065CC1343CB60BFF34F8FFEE700BF00ED00E02F
S315080065DC0400FA0580B500AF024B9847024B984762
S315080065EC00BF80BD216600086D68000880B500AF45
S315080065FC024B9847024B984700BF80BDB56600080A
S3150800660C9569000880B500AF014B984700BF80BD5F
S3150800661CB965000880B586B000AF01214FF400308B
S3150800662C1A4B984701210520194B98471823FB75D7
S3150800663C0423BB820323BB7507F1140319461548BB
S3150800664C154B98470423FB750823BB8207F11403E3
S3150800665C19461048104B98474FF461437B6000234A
S3150800666C3B8100237B810023BB8100233B820C23C7
S3150800667CFB813B1D19460948094B984701210748D8
S3150800668C084B984700BF1837BD4680BD997300085C
S3150800669C5D730008000801406D6F00080044004057
S315080066AC117400088975000880B500AF254B1B7856
S315080066BC002B15D12448254B98470346012B3FD16F
S315080066CC214B1B78002B3BD0214B98470246214B7C
S315080066DC1A601C4B01221A701F4B00221A702FE0ED
S315080066EC1D4B1B780133184A13441846174B984709
S315080066FC0346012B19D1184B1B780133DAB2164B0A
S3150800670C1A70114B1A78144B1B789A4218D10D4BE8
S3150800671C00221A700C4B5B78FF2B11D10A4B9B7815
S3150800672C002B0DD10D4B98470AE0094B98470246AA
S3150800673C084B1B6864339A4202D9024B00221A7022
S3150800674C00BF80BD20000020240000206D670008D3
S3150800675C81650008680000206C000020116600089E
S3150800676C80B582B000AF786020210A480A4B98475A
S3150800677C0346012B08D10748084B98470346DAB25B
S3150800678C7B681A70012300E0002318460837BD46BB
S3150800679C80BD00BF00440040E9750008C9750008B3
S315080067AC80B487B000AFB9607A603B600346FB8162
S315080067BC0023FB7548E0FA89FB7D284911F813304C
S315080067CC1846FB7D25495B000B445B780344013373
S315080067DC03FB02F348F6A04292FBF3F103FB01F329
S315080067ECD31A002B2DD1FA89FB7D1C4911F81330CD
S315080067FC1846FB7D19495B000B445B78034401334F
S3150800680C03FB02F348F6A04292FBF3F39AB2BB6879
S3150800681C1A80BB681B88002B13D0BB681B88B3F582
S3150800682C806F0ED8FB7D0D4A12F813207B681A7000
S3150800683CFB7D0A4A5B0013445A783B681A7001239D
S3150800684C06E0FB7D0133FB75FB7D112BB3D90023C9
S3150800685C18461C37BD4680BC704700BF207600081A
S3150800686C90B58BB000AF012101203C4B9847012114
S3150800687C08203A4B98474FF48073BB84482387F813
S3150800688C273007F1240319463548364B98474FF4F9
S3150800689C0073BB84182387F82730032387F8263020
S315080068AC07F1240319462E482E4B984701214FF41D
S315080068BCEA102D4B984701214FF000702B4B984747
S315080068CC2B482C4B984707F1180318462A4B984720
S315080068DC3B1D7A1DB91D4FF4FA70284CA0470023AE
S315080068ECBB770023FB77002387F82030002387F833
S315080068FC2130002387F82230002387F82330002321
S3150800690CBB760023FB767B79013BDBB23B773B7985
S3150800691C013BDBB27B77FB883B8307F118031946EF
S3150800692C1348174B98470023BB740023FB740123A9
S3150800693C3B7500233B8100237B810023BB8100230D
S3150800694CFB8100233B8201237B7507F1080318465C
S3150800695C0C4B984700BF2C37BD4690BD5D7300089D
S3150800696C000C01406D6F00081D7100089973000832
S3150800697C00640040FD6900085D6D0008AD670008FD
S3150800698C496A0008E96B000880B586B000AF002399
S3150800699CFB7500211248134B98470346002B1AD057
S315080069AC3B461A4600210E480F4B98473B7A002B5C
S315080069BC06D13B6840F26762934201D10123FB750D
S315080069CCFB7D012B07D1FB7AFF2B04D13B7B002BDC
S315080069DC01D1064B984700BF1837BD4680BD00BF8E
S315080069EC00640040256F0008B16D000811660008A8
S315080069FC80B582B000AF78607B680E4A93420AD1A4
S31508006A0C01214FF000700C4B984700214FF0007095
S31508006A1C094B984709E001214FF08060064B9847CF
S31508006A2C00214FF08060044B984700BF0837BD46DD
S31508006A3C80BD00BF00640040D573000880B485B0E3
S31508006A4C00AF786039600023FB730023BB607B685A
S31508006A5C1B6823F002027B681A607B681B6843F08C
S31508006A6C01027B681A6002E0BB680133BB607B6875
S31508006A7C5B6803F00103002B04D1BB684FF6FF7269
S31508006A8C9342F1D17B685B6803F00103002B02D1BA
S31508006A9C0023FB739CE03B689B79012B06D17B6832
S31508006AAC1B6843F080027B681A6005E07B681B68EC
S31508006ABC23F080027B681A603B68DB79012B06D1D0
S31508006ACC7B681B6843F040027B681A6005E07B68AC
S31508006ADC1B6823F040027B681A603B681B7A012B03
S31508006AEC06D17B681B6843F020027B681A6005E0B8
S31508006AFC7B681B6823F020027B681A603B685B7A0C
S31508006B0C012B06D17B681B6843F010027B681A6060
S31508006B1C05E07B681B6823F010027B681A603B68EB
S31508006B2C9B7A012B06D17B681B6843F008027B68AD
S31508006B3C1A6005E07B681B6823F008027B681A60FC
S31508006B4C3B68DB7A012B06D17B681B6843F0040291
S31508006B5C7B681A6005E07B681B6823F004027B6877
S31508006B6C1A603B689B789A073B68DB781B061A43C6
S31508006B7C3B681B791B041A433B685B791B051A4354
S31508006B8C3B681B88013B1A437B68DA617B681B6888
S31508006B9C23F001027B681A600023BB6002E0BB6825
S31508006BAC0133BB607B685B6803F00103002B04D0E0
S31508006BBCBB684FF6FF729342F1D17B685B6803F0B2
S31508006BCC0103002B02D00023FB7301E00123FB73A6
S31508006BDCFB7B18461437BD4680BC704780B485B01D
S31508006BEC00AF78600023FB607B689B7A1A4601230A
S31508006BFC9340FB60554A554BD3F8003243F00103DA
S31508006C0CC2F800325149514BD3F81C22FB68DB43BE
S31508006C1C1340C1F81C327B681B7B002B25D14B49D2
S31508006C2C4A4BD3F80C22FB68DB431340C1F80C32F1
S31508006C3C46497B689B7A18467B68DB881B047A680E
S31508006C4C52881A4300F1480341F833203F497B68C0
S31508006C5C9B7A18467B689B881B047A6812881A43A9
S31508006C6C00F14803DB000B445A607B681B7B012B45
S31508006C7C24D13649354BD3F80C22FB681343C1F89B
S31508006C8C0C3232497B689B7A18467B681B881B0436
S31508006C9C7A6852881A4300F1480341F833202B4985
S31508006CAC7B689B7A18467B689B881B047A68D28813
S31508006CBC1A4300F14803DB000B445A607B68DB7A05
S31508006CCC002B09D12149214BD3F80422FB68DB435D
S31508006CDC1340C1F8043207E01C491C4BD3F80422B4
S31508006CECFB681343C1F804327B681B89002B08D157
S31508006CFC1649164BD3F81422FB68DB431340C1F82C
S31508006D0C14327B681B89012B07D110490F4BD3F81A
S31508006D1C1422FB681343C1F814327B685B7B012B86
S31508006D2C07D10A49094BD3F81C22FB681343C1F84F
S31508006D3C1C32064A054BD3F8003223F00103C2F87D
S31508006D4C003200BF1437BD4680BC70470064004053
S31508006D5C80B483B000AF78607B6800229A717B6838
S31508006D6C0022DA717B6800221A727B6800225A723A
S31508006D7C7B6800229A727B680022DA727B68002292
S31508006D8C9A707B680022DA707B6803221A717B681A
S31508006D9C02225A717B6801221A8000BF0C37BD4645
S31508006DAC80BC704780B485B000AFF8600B467A603B
S31508006DBCFB72FB7AFA681B331B0113441B68DBB2A4
S31508006DCC03F00403DAB27B681A727B681B7A002B11
S31508006DDC09D1FB7AFA681B331B0113441B685A0D3D
S31508006DEC7B681A6008E0FB7AFA681B331B011344AC
S31508006DFC1B68DA087B685A60FB7AFA681B331B0136
S31508006E0C13441B68DBB203F00203DAB27B685A72CE
S31508006E1CFB7AFA681B331B01134404331B68DBB279
S31508006E2C03F00F03DAB27B689A72FB7AFA681B33A3
S31508006E3C1B01134404331B681B0ADAB27B68DA7429
S31508006E4CFB7AFA681B01134403F5DC731B68DAB288
S31508006E5C7B68DA72FB7AFA681B01134403F5DC7358
S31508006E6C1B681B0ADAB27B681A73FB7AFA681B0171
S31508006E7C134403F5DC731B681B0CDAB27B685A7374
S31508006E8CFB7AFA681B01134403F5DC731B681B0EAB
S31508006E9CDAB27B689A73FB7AFA681B01134403F51A
S31508006EACDE731B68DAB27B68DA73FB7AFA681B0145
S31508006EBC134403F5DE731B681B0ADAB27B681A7473
S31508006ECCFB7AFA681B01134403F5DE731B681B0C6B
S31508006EDCDAB27B685A74FB7AFA681B01134403F519
S31508006EECDE731B681B0EDAB27B689A74FB7A002B6E
S31508006EFC06D1FB68DB6843F02002FB68DA6005E024
S31508006F0CFB681B6943F02002FB681A6100BF143743
S31508006F1CBD4680BC704700BF80B485B000AF7860B2
S31508006F2C0B46FB700023FB73FB78002B06D17B68A2
S31508006F3CDB68DBB203F00303FB730BE0FB78012B76
S31508006F4C06D17B681B69DBB203F00303FB7301E014
S31508006F5C0023FB73FB7B18461437BD4680BC704771
S31508006F6C80B489B000AF786039600023FB610023D8
S31508006F7C3B610023BB610023FB6000237B6100237C
S31508006F8CBB603B68DB7803F00F03FB613B68DB787F
S31508006F9C03F01003002B05D03B689B781A46FB6957
S31508006FAC1343FB613B681B88DBB2002B44D07B6820
S31508006FBC1B687B610023BB6138E00122BB6902FABE
S31508006FCC03F3FB603B681B881A46FB6813403B615E
S31508006FDC3A69FB689A4226D1BB699B00FB600F2273
S31508006FECFB6802FA03F3BB60BB68DB437A691340A0
S31508006FFC7B61FA69FB6802FA03F37A6913437B61CE
S3150800700C3B68DB78282B05D10122BB699A407B6843
S3150800701C5A6108E03B68DB78482B04D10122BB692E
S3150800702C9A407B681A61BB690133BB61BB69072B44
S3150800703CC3D97B687A691A603B681B88FF2B46D9CB
S3150800704C7B685B687B610023BB613AE0BB690833EC
S3150800705C012202FA03F3FB603B681B881A46FB689D
S3150800706C13403B613A69FB689A4227D1BB699B007E
S3150800707CFB600F22FB6802FA03F3BB60BB68DB43B9
S3150800708C7A6913407B61FA69FB6802FA03F37A6939
S3150800709C13437B613B68DB78282B05D1BB69083326
S315080070AC01229A407B685A613B68DB78482B05D1EC
S315080070BCBB69083301229A407B681A61BB690133A4
S315080070CCBB61BB69072BC1D97B687A695A6000BF5B
S315080070DC2437BD4680BC704780B483B000AF786057
S315080070EC0B467B807A887B681A6100BF0C37BD46D5
S315080070FC80BC704780B483B000AF78600B467B8049
S3150800710C7A887B685A6100BF0C37BD4680BC7047CD
S3150800711C80B487B000AF78600B46FB7000233B61E8
S3150800712C0023FB6000237B610023BB607B68002B7C
S3150800713C03DA2E4BDB697B6102E02C4B5B687B61C7
S3150800714C7B681B0C03F00F03BB607B689BB23B612F
S3150800715C7B6803F44013B3F5401F0AD17B6923F00F
S3150800716C70637B61214A214B5B6823F07063536023
S3150800717C21E07B6803F48013002B0ED00322BB6836
S3150800718C02FA03F3FB60FB68DB437A6913407B6105
S3150800719C7B6943F070637B610DE07B685B0D1B01BB
S315080071AC3A6902FA03F3DB437A6913407B617B691C
S315080071BC43F070637B61FB78002B08D07B685B0D12
S315080071CC1B013A6902FA03F37A6913437B617B68FC
S315080071DC002B03DA054A7B69D36102E0034A7B6913
S315080071EC536000BF1C37BD4680BC70470000014089
S315080071FC80B487B000AF786000237B6100233B61C5
S3150800720C0023FB600023BB604C4B5B6803F00C034C
S3150800721C7B617B69042B07D0082B09D0002B33D153
S3150800722C7B68474A1A6033E07B68454A1A602FE048
S3150800723C424B5B6803F470133B61404B5B6803F489
S3150800724C8033FB603B699B0C02333B61FB68002B6C
S3150800725C06D13B693B4A02FB03F27B681A6017E0CE
S3150800726C364B5B6803F40033002B06D03B69354A72
S3150800727C02FB03F27B681A600AE03B69304A02FBA0
S3150800728C03F27B681A6003E07B682D4A1A6000BF1C
S3150800729C2A4B5B6803F0F0037B617B691B097B61F6
S315080072AC294A7B6913441B78DBB2BB607B681A6876
S315080072BCBB68DA407B685A60204B5B6803F4E06372
S315080072CC7B617B691B0A7B611F4A7B6913441B78AC
S315080072DCDBB2BB607B685A68BB68DA407B689A602D
S315080072EC164B5B6803F460537B617B69DB0A7B6135
S315080072FC154A7B6913441B78DBB2BB607B685A68FA
S3150800730CBB68DA407B68DA600C4B5B6803F4404375
S3150800731C7B617B699B0B7B610C4A7B6913441B78ED
S3150800732CDBB2BB607B68DA68BB68B2FBF3F27B68DE
S3150800733C1A6100BF1C37BD4680BC7047001002405E
S3150800734C00127A0000093D00000000201000002001
S3150800735C80B483B000AF78600B46FB70FB78002BCB
S3150800736C06D00949084B9A697B6813438B6106E07A
S3150800737C0549054B9A697B68DB4313408B6100BF53
S3150800738C0C37BD4680BC70470010024080B483B0F1
S3150800739C00AF78600B46FB70FB78002B06D00949CA
S315080073AC084BDA697B681343CB6106E00549054B44
S315080073BCDA697B68DB431340CB6100BF0C37BD46EB
S315080073CC80BC70470010024080B483B000AF786070
S315080073DC0B46FB70FB78002B06D00949084B1A693B
S315080073EC7B6813430B6106E00549054B1A697B68F4
S315080073FCDB4313400B6100BF0C37BD4680BC70479E
S3150800740C0010024080B58CB000AF7860396000235C
S3150800741CFB620023BB6200237B6200233B620023D2
S3150800742CFB617B68FB617B681B8A9BB2FB62FA6A11
S3150800743C4CF6FF731340FB623B68DB881A46FB6A03
S3150800744C1343FB62FB6A9AB27B681A827B689B8938
S3150800745C9BB2FB62FA6A4EF6F3131340FB623B6867
S3150800746C9A883B681B8913439AB23B685B8913431A
S3150800747C9BB21A46FB6A1343FB62FB6A9AB27B6899
S3150800748C9A817B689B8A9BB2FB62FA6A4FF6FF432A
S3150800749C1340FB623B689B891A46FB6A1343FB62E3
S315080074ACFB6A9AB27B689A8207F108031846304B36
S315080074BC9847FB692F4A934202D17B69BB6201E06C
S315080074CC3B69BB627B689B899BB21BB2002B0CDAAF
S315080074DCBA6A13469B0013449A001A443B681B6805
S315080074EC5B00B2FBF3F37B620BE0BA6A13469B00B4
S315080074FC13449A001A443B681B689B00B2FBF3F3CF
S3150800750C7B627B6A1C4AA2FB03235B091B01FB6299
S3150800751CFB6A1B09642202FB03F37A6AD31A3B62E1
S3150800752C7B689B899BB21BB2002B0CDA3B6ADB008F
S3150800753C3233114AA2FB03235B0903F00703FA6AE9
S3150800754C1343FB620BE03B6A1B0132330A4AA2FB6C
S3150800755C03235B0903F00F03FA6A1343FB62FB6A06
S3150800756C9AB27B681A8100BF3037BD4680BD00BF12
S3150800757CFD710008003801401F85EB5180B483B0BB
S3150800758C00AF78600B46FB70FB78002B08D07B6845
S3150800759C9B899BB243F400539AB27B689A8107E0A5
S315080075AC7B689B899BB223F400539AB27B689A81B9
S315080075BC00BF0C37BD4680BC704700BF80B483B093
S315080075CC00AF78607B689B889BB2C3F308039BB2B9
S315080075DC18460C37BD4680BC704700BF80B485B0D2
S315080075EC00AF78600B467B800023FB737B681B8897
S315080075FC9AB27B8813409BB2002B02D00123FB73F3
S3150800760C01E00023FB73FB7B18461437BD4680BC90
S3090800761C704700BFE6
S3150800762005020602060307030803090309040A04F8
S315080076300B040C040C050D050E050F050F061006A8
S309080076401007100809
S3150800764400000000010203040102030406070809F6
S309080076540204060810
S705080061FB96
